:100000000C94F2020C9439030C9439030C943903C8
:100010000C9439030C9439030C9439030C94390370
:100020000C9439030C9439030C94BE280C94902939
:100030000C94251F0C9439030C9439030C94390348
:100040000C9439030C9439030C9439030C94390340
:100050000C9439030C948D1F0C9439030C943903C0
:100060000C9439030C9439030C9439030C94390320
:100070000C9439030C9439030C9439030C94390310
:100080000C9439030C9439030C9439030C94390300
:100090000C9439030C9439030C9439030C943903F0
:1000A0000C9439030C9439030C943903AB05AD055A
:1000B000B805AF05B105B305B505B705BA05BC056B
:1000C000BE05C905C005C205C405C605C805CB05E2
:1000D000A614A614D814D81416153615CB16CB169C
:1000E0007815CB16251625169716A016CB16C4160E
:1000F00032163216321632163216321632163216C0
:1001000032163216321632163216321632163216AF
:100110004316511658165F1669165A175A176C1758
:100120006C1763176C176C176C175A175A176817E8
:100130006C176C176817FD29242A162B242A162BF6
:10014000702A932A162BE92AF82A07634236B79BAE
:10015000D8A71A39685618AEBAAB558C1D3CB7CC27
:100160005763BD6DEDFD753EF6177231BF0000009F
:10017000803F05A84CCDB2D44EB93836A9020C50F8
:10018000B9918688083CA6AAAA2ABE000000803F32
:1001900029001E001F00200021002200230024004F
:1001A0002500260027002D002E00310035002B00F1
:1001B000000014001A000800150017001C001800A9
:1001C0000C00120013002F0030002A00E000000095
:1001D00004001600070009000A000B000D000E00C5
:1001E0000F003300340028000000E10000001D0073
:1001F0001B00060019000500110010003600370032
:1002000038000000E50001510151E2000000E30068
:100210002C0000002C0000002C000000E700E6008D
:100220000000E400025100003A003B003C003D00A9
:100230003E003F00400041004200430044004500B2
:1002400049004C0039000000C25CC35CC55CC65C60
:10025000C75CC85CC95CCA5C47004800520000002B
:100260000000E0000000810080007F00000000002E
:10027000000000004A004B0050004F00000000004A
:10028000E10000003502CB5CCC5C00000000000007
:1002900000004D004E005100000000000100010070
:1002A000E2000000E3000000000000000000000089
:1002B00000000000000000000000010000003A0003
:1002C0003B003C003D003E003F004000410042003A
:1002D00043004400450049004C0039000000C25C66
:1002E000C35CC55CC65CC75CC85CC95CCA5C4700D3
:1002F000480052000000005C00000000BC00AE009E
:10030000BB0000000000000000004A004B0050004D
:100310004F0000000000000000003502CB5CCC5C08
:1003200000000000000000004D004E0051000000E1
:1003300000000000000000000000000000000000BD
:1003400000000000000000000000000000000000AD
:10035000010000047F3F1F643214643214783C1E95
:100360001E140A056801F000B40078005A0000006D
:10037000000000010101010101010101020202026C
:10038000020202020203030303030303030404043F
:100390000404040505050505060606060607070705
:1003A00007080808080909090A0A0A0A0B0B0B0CB6
:1003B0000C0C0D0D0D0E0E0F0F0F10101111111250
:1003C0001213131414151516161717181819191ACD
:1003D0001A1B1C1C1D1D1E1F1F202021222223242E
:1003E000252526272728292A2B2B2C2D2E2F2F3069
:1003F000313233343536363738393A3B3C3D3E3F7F
:100400004041424344464748494A4B4C4D4F505166
:100410005253555657585A5B5C5E5F606263646620
:1004200067696A6C6D6E707173747678797B7C7EA7
:100430008081838486888A8B8D8F91929496989AF6
:100440009B9D9FA1A3A5A7A9ABADAFB1B3B5B7B90C
:10045000BBBDBFC1C4C6C8CACCCFD1D3D6D8DADCE5
:10046000DFE1E4E6E8EBEDF0F2F5F7FAFCFF040378
:10047000300000000A0344005A003600300000003B
:1004800010034B0042004400460061006E00730000
:1004900000000403090409023B00020100A0FA095C
:1004A00004000001030101000921110100012240A3
:1004B000000705810308000A090401000103000088
:1004C0000009211101000122C0000705820320005C
:1004D0000A1201100100000008EDFE602201000177
:1004E00002030105010902A10185020901A100051C
:1004F0000919012905150025019505750181029548
:1005000001750381010501093009311581257F95A8
:10051000027508810609381581257F9501750881C6
:1005200006050C0A38021581257F9501750881069C
:10053000C0C005010980A101850316010026030042
:100540001A81002A8300751095018100C0050C09ED
:1005500001A1018504160100269C021A01002A9CB3
:1005600002751095018100C005010906A1018505EC
:10057000050719E029E71500250195087501810295
:100580000508190129059505750191029501750365
:1005900091010507190029EF1500250195F0750156
:1005A0008102C005010906A101050719E029E71527
:1005B00000250195087501810295017508810105E5
:1005C0000819012905950575019102950175039199
:1005D000010507190029FF150026FF00950675087B
:1005E0008100C00011241FBECFEFDAE0DEBFCDBF17
:1005F00004B603FE27C08091970290919802A091C3
:100600009902B0919A028730904BA740B04BD1F439
:1006100010929702109298021092990210929A02E8
:1006200014BE84B7877F84BF0FB6F894A8958091D5
:100630006000886180936000109260000FBEE0E06F
:10064000F8E3099511E0A0E0B1E0E8ECFEE502C0B6
:1006500005900D92A633B107D9F722E0A6E3B1E0E9
:1006600001C01D92A739B207E1F70E94E0250C9462
:10067000622F0C9400000C942B09229A2A9A089558
:100680000E942A090C943D0381FF02C02A9801C0F0
:100690002A9A0C94010481E0089581E008950C9455
:1006A0004D031F93CF93DF9300D000D01F92CDB79F
:1006B000DEB749835A832091850189819A8121116E
:1006C00012C0662349F00E947F1C182F682F898171
:1006D0009A810E94241C03C00E94531C182F698118
:1006E0007A81812F04C00E947F1C69817A810F90DA
:1006F0000F900F900F900F90DF91CF911F910C945E
:100700007D06FC01408151816281738184810C945A
:1007100051030C943B03CF92DF92EF92FF9286300D
:1007200030F4811105C0909180009F7D04C085E068
:1007300090918000906290938000282F30E0AFEF7E
:10074000BFEF0E94F32E25E030E040E050E00E9431
:10075000CB2E2C3784E138074105510530F4C9010F
:1007600069E070E00E94A32E29C0DA01C9018A5015
:10077000974DAF4FBF4F6627782F892F9A2F25EFC0
:1007800038E241E050E00E94CB2E69017A01CA01B3
:10079000B9010E94932E9B01AC01C701B6010E94D2
:1007A000932EBB27A92F982F872F009721E0A20710
:1007B000B10511F0BC0102C06FEF7FEF70938B00A9
:1007C00060938A00FF90EF90DF90CF900895269A73
:1007D0002E9882E28093800089E1809381008FEFE0
:1007E0009FEF90938700809386000C9460230E9473
:1007F000AF1D811102C00E943C1E0E94E7030C94B1
:10080000400308950C94440308950E944A170E94DF
:1008100004042FEF84E39CE0215080409040E1F7F6
:1008200000C000000C94B31F0F931F93CF93DF936E
:100830008C010E948103EC01B8010E944F038823C0
:1008400009F451C2CC3C8CE5D80709F4E1C0E8F5C5
:10085000C43CECE5DE0709F4A5C0F8F4C5318CE52D
:10086000D80778F4C2309CE5D90708F052C1C11509
:10087000ECE5DE0709F467C0C130DC4509F46BC064
:1008800026C2C23C8CE5D80709F478C008F07EC0C7
:10089000C631DC4509F4F4C11AC2F8018281C83CB2
:1008A000FCE5DF0709F49CC040F4C63CECE5DE073C
:1008B00009F48AC008F482C08DC0CA3C9CE5D907FF
:1008C00009F49AC008F492C09DC0C43DFCE5DF075E
:1008D00009F4F8C0C0F4F8018281C03DFCE5DF07EF
:1008E00009F4BFC040F4CE3CECE5DE0709F49DC03E
:1008F00008F496C0A8C0C23D9CE5D90709F4CFC052
:1009000008F4BFC0DAC0C93DFCE5DF0709F49DC1AA
:1009100060F4C73D9CE5D90709F44DC108F06EC1EC
:10092000C53DDC4509F4DEC0D2C1CD3D8CE5D8071C
:1009300009F4E6C0CE3D9CE5D907C1F0CC3DDC45CD
:1009400009F0C5C1D6C0F8018281882309F4CBC162
:100950000E940504C8C1F8018281882309F4C3C13B
:1009600080911D02816080931D02BDC1F8018281CA
:10097000882309F4B8C10E943C1EB5C1F8018281E8
:10098000882309F4B0C10E94F20DADC1F801828143
:10099000882309F4A8C10E94FF1C827261F00E94A2
:1009A0008E0DA1C1F8018281882309F49CC10E94A7
:1009B000FF1C8272A1F30E94800D95C1882309F467
:1009C00092C10E94830C8FC1882309F48CC10E94BC
:1009D000A70C89C1882309F486C10E94C70C83C172
:1009E000882309F480C10E94E70C7DC1882309F4A3
:1009F0007AC10E94070D77C1882309F474C10E944F
:100A0000270D71C1882309F46EC10E94360B6BC19A
:100A1000F8018281882309F466C10E944B0B63C1EF
:100A2000882309F460C181E029C0882309F45BC1EF
:100A30000E942D0B823028F00E942D0B853008F487
:100A4000BACF82E01BC0882309F44DC10E942D0B50
:100A5000863028F00E942D0B883008F4ACCF86E059
:100A60000DC0882309F43FC10E942D0B893028F066
:100A70000E942D0B8E3008F49ECF89E00E94910DCC
:100A800032C1882309F42FC10E942D0B8F3028F02A
:100A90000E942D0B843108F48ECF8FE0EFCF882396
:100AA00009F421C10E942D0B853128F00E942D0BE5
:100AB000873108F480CF85E1E1CF882309F413C1A1
:100AC00088E1DCCFF8018281882309F40CC10E94FF
:100AD0002D0B893128F00E942D0B823208F46BCF48
:100AE00089E1CCCFF8018281882309F4FCC083E23C
:100AF000C5CFF8018281882309F4F5C080E006C0E3
:100B0000F8018281882309F4EEC082E00E948126E8
:100B1000EAC0F8018281882309F4DEC00E94AF1D7B
:100B2000811102C00E943C1E0E94CC1D90E0909357
:100B3000880280938702FE01E350FC45E231F10513
:100B400030F4EA5AFF4F809187020C94ED2E809189
:100B50008702816027C0826025C0846023C08061D5
:100B600021C080621FC080641DC080681BC084607B
:100B7000886018C08E7F16C08D7F14C08B7F12C016
:100B80008F7E10C08F7D0EC08F7B0CC08F770AC008
:100B90008B7F877F07C087FB222720F991E0922770
:100BA00090FB87F980938702809187020E94D01D75
:100BB0000E944A1798C0F8018281882351F0109250
:100BC0003B010E94571F909338018093370182E0C8
:100BD00022C080913B0181110FC08091370190911B
:100BE00038010E94631F883C910530F486E20E9420
:100BF000DC1286E20E94FA1382E024C0F8018281AE
:100C0000882361F010923C010E94571F90933A0193
:100C10008093390180E20E94621465C080913C019A
:100C200081110FC08091390190913A010E94631F98
:100C3000883C910530F487E20E94DC1287E20E9432
:100C4000FA1380E20E9469144EC0F801828181117A
:100C5000D9CF80913C018111F4CF809139019091DD
:100C60003A010E94631F883C910558F780E20E9478
:100C7000691488E20E94DC1288E20E94FA1333C0F1
:100C80000E94FF1C282FF801828140910E01509193
:100C90000F01882379F02A7A91E009F490E090938B
:100CA0003601911102C069E201C065E3CA010E94E8
:100CB000A31E0AC080913601811102C069E201C001
:100CC00065E3CA010E94AE1E0E944B1D0CC081E06C
:100CD00080933B0180933C01C801DF91CF911F912C
:100CE0000F910C944B0380E0DF91CF911F910F91F6
:100CF000089580E090E0089508959FE0799FF001C5
:100D000011249BE4899FE00DF11D1124E60FF11DD4
:100D1000EE0FFF1FE057FE4F859194910895880FC5
:100D2000991FFC01EE5AFC4F859194910895CF9341
:100D3000DF930E947D060E948A08EC01811521E55F
:100D4000920708F042C0811560E5960708F031C1AE
:100D5000883E910500F5803E910508F0D7C1883A9C
:100D6000910570F4853A910508F0A6C0813091058F
:100D700009F4CCC108F47DC1049708F0C7C179C15A
:100D80008F3B910508F4A3C0803C910508F471C124
:100D9000805C9109FDC0C11580E3D80780F4C115BE
:100DA00090E2D90708F0F2C0C03FD10508F461C154
:100DB000CF3FD10511F008F0A9C1D065A7C1C11579
:100DC00020E4D20708F0F2C0E7C0811569E5960774
:100DD00060F5C11588E5D80708F037C1C11594E55D
:100DE000D90778F4C11523E5D20708F013C1C1155E
:100DF00062E5D60708F0F8C0DC2FCC27C16FD06AB7
:100E000085C1C11585E5D80708F41AC1C11596E555
:100E1000D90708F02EC18C2F0E9407098F71C82FA7
:100E2000D0E0DC2FCC27D06271C18D3B2CE592073E
:100E300009F416C1F0F4CB3B8CE5D80709F40AC1DC
:100E400008F00BC1C1152AE5D20708F012C18C2F9A
:100E50008F700E94070994E0D695C7959A95E1F79F
:100E6000CF70D0E0DC2FCC27D06A8F70806EC82B7B
:100E70004DC1803C9C4509F4F9C0C13C8CE5D807C4
:100E800060F4CE3B9CE5D90709F4EDC0CF3BDC45CF
:100E900009F0EFC0C0E0D2ED39C1CE019056811506
:100EA000904208F0E6C08D2F8F710E940709DD2760
:100EB000D0628F71D82B2AC1853A910509F4DCC024
:100EC000863A910509F0DBC0C2E8D0E41FC1883A38
:100ED000910509F4D7C0893A910509F4D6C08A3A38
:100EE000910509F4D5C08B3A910509F4D4C08C3A28
:100EF000910509F4D3C08B3B910509F4D2C08C3B1A
:100F0000910509F4D1C08D3A910509F4D0C0803B18
:100F1000910509F4CFC08E3A910509F4CEC08F3AFD
:100F2000910509F4CDC0813B910509F4CCC0823B09
:100F3000910509F4CBC0833B910509F4CAC0843BF9
:100F4000910509F4C9C0853B910509F4C8C0863BE9
:100F5000910509F4C7C0873B910509F4C6C0883BD9
:100F6000910509F4C5C0893B910509F4C4C08D3BC6
:100F7000910509F4C3C08E3B910509F4C2C08A3BB8
:100F8000910509F4C1C0C0E0D4E4C0C0CE019F7097
:100F90000E948F06EC01BAC0CE019927D3FF03C08F
:100FA000EC01D86CB3C0EC01D06CB0C0DF70D06A7B
:100FB000ADC0837021E030E002C0220F331F8A955C
:100FC000E2F73C68CE0174E0969587957A95E1F753
:100FD0008370382BCF70C695C69580E2C89FE0011C
:100FE0001124C22BD32B92C04C2F4695469590E2EC
:100FF000499FA0011124C370DD2721E030E0C90121
:1010000002C0880F991FCA95E2F7EC01C42BD52BBB
:10101000DC687CC04C2F4695469580E2489FA00135
:101020001124C370DD2721E030E0C90102C0880F20
:10103000991FCA95E2F7EC01C42BD52BDA6866C07C
:10104000DC2FCC27C46FD06A61C0DC2FCC27C06FE7
:10105000D06A5CC0C0E0D4ED59C0C0E0D5ED56C048
:10106000C0E0D1ED53C0C0E0D0ED50C0C0E0D3ED42
:101070004DC0C0E0D0E04AC0C1E8D0E447C0C3E8FA
:10108000D0E444C0C2EED4E441C0C9EED4E43EC0D2
:10109000CAEED4E43BC0C5EBD4E438C0C6EBD4E41C
:1010A00035C0C3EBD4E432C0C4EBD4E42FC0C7EBEB
:1010B000D4E42CC0CCECD4E429C0CDECD4E426C0DC
:1010C000C3E8D5E423C0CAE8D5E420C0C2E9D5E42A
:1010D0001DC0C4E9D5E41AC0C1E2D6E417C0C3E21A
:1010E000D6E414C0C4E2D6E411C0C5E2D6E40EC012
:1010F000C6E2D6E40BC0C7E2D6E408C0CFE6D4E42B
:1011000005C0C0E7D4E402C0CAE2D6E4CE01DF9154
:10111000CF9108958238910549F1B0F4813391055A
:1011200009F458C048F48932910509F44EC08A3256
:10113000910509F454C008958533910509F440C020
:101140008933910599F00895833E910529F138F48A
:10115000803E910591F0823E9105A1F00895863E72
:101160009105F9F0873E910531F1089520918702AC
:1011700020FD3AC021FD38C008958091870280FD8E
:1011800035C032C08091870282FF32C080918702D1
:1011900084FD30C083EE39C08091870282FD28C073
:1011A000F5CF8091870283FF27C08091870284FD5D
:1011B00021C087EE2AC08091870283FD1DC0F5CF34
:1011C0008091870285FD1AC01BC08091870285FD32
:1011D00017C014C08091870286FD14C015C080918D
:1011E000870286FD11C00EC080EE0FC089E30DC0DE
:1011F00082EE0BC080E009C086EE07C089E205C020
:1012000085E303C08AE201C081E390E008959091F4
:10121000870292FF0DC0282F2871283019F4877F8C
:10122000846006C0282F2471243011F48B7F8860DD
:1012300093FF0DC0282F2871283119F4877E84610F
:1012400006C0282F2471243111F48B7E886194FD0F
:10125000877E089508950895E82FF0E0EE0FFF1FB0
:10126000E35CFE4F8081918108950895E0E3F1E011
:1012700041E050E025E02E0F9191A92FA295AF708B
:10128000B0E091963C9191979F70BA0102C0660FB1
:10129000771F9A95E2F7CB018095832391968C93E3
:1012A0002E13EACFA1E2B1E041E050E02FE02A0F97
:1012B0008D91E82FE295EF70F0E031A18F70BA01C7
:1012C00002C0660F771F8A95E2F7CB01962F9095A3
:1012D000932391A392A1892B82A32A13E9CFE7E458
:1012E000F1E0ADE3B1E0119211921D921D9271E017
:1012F000E135F707C1F785E00E94180A0C94F7035F
:101300004F925F927F928F929F92AF92BF92CF92B5
:10131000DF92EF92FF920F931F93CF93DF9320E31F
:10132000422E21E0522EA7E4B1E020E001E010E0DF
:101330005D018D909C90119711961C921E92E20176
:1013400089912E01E82FE295EF70F0E031A18F70C6
:10135000A80102C0440F551F8A95E2F7CA01342B39
:1013600031A342A1382F3095432342A350EA5A9526
:10137000F1F791E2C92E91E0D92E40E050E0E6016C
:1013800079906E01672D62956F7070E0EB01E8A0B7
:101390006D917C911197F12CD72DDF7002C0F594DF
:1013A000E794DA95E2F7E0FC08C07801042E02C069
:1013B000EE0CFF1C0A94E2F702C0E12CF12C6E291E
:1013C0007F2911967C936E934F5F5F4F4F3051058D
:1013D000B1F691A1392331A392A1892B82A3129650
:1013E00081E0F501408151818416950609F480E081
:1013F000282BF1E0A135BF0709F09ACF45E06DE356
:1014000071E087E491E00E94190A0E94890381E05B
:10141000DF91CF911F910F91FF90EF90DF90CF90D0
:10142000BF90AF909F908F907F905F904F90089566
:101430000895FF920F931F93CF93DF93F82E092FF8
:10144000162FD72FC42F222349F081E08093530118
:101450000E94571F90935201809351018091530134
:101460008823D9F080915101909152010E94631F0D
:10147000069798F0EF2DF02FA12FBD2F80E090E080
:101480004C2F50E08417950734F4219131912D931E
:101490003D930196F7CF10925301DF91CF911F91A9
:1014A0000F91FF900895EF92FF920F931F93CF93A8
:1014B000DF93E901662309F44BC0242F30E0EFEFFE
:1014C000F0E0E61BF109B901E69F9001E79F300DBE
:1014D000F69F300D1124232F8B01031B11095CE3B0
:1014E000E52EF12CB7010E94A32EFB01BC01069F43
:1014F000C001079F900D169F900D1124B7010E9407
:10150000A32EE230F105B1F040F4309779F0319735
:1015100011F5832F242F461B21C0E430F105A1F0E3
:1015200068F03597C1F4842F861B18C0832F262FAF
:10153000230F14C0862F830FE42F03C0E42FE61B74
:10154000842F432F2E2F0AC0842F462F430F06C00F
:10155000842F242F03C080E020E040E0E42FF0E05F
:10156000E259FC4F4491E22FF0E0E259FC4F949194
:10157000E82FF0E0E259FC4FE49149839883EA8335
:10158000DF91CF911F910F91FF90EF90089580917F
:101590004C02282F26952F7330E02115310519F4C0
:1015A0008178826005C02532310524F08178886415
:1015B00080934C0230914C02432F441F4427441F18
:1015C00020914D02522F550F852F842B27FB9927F1
:1015D00090F9893641E094077CF068E671E00E945A
:1015E000B72E80FB37F930934C0286952078822BFA
:1015F00090FB87F980934D02089588E090E00C9469
:10160000222FCF93DF9300D000D0CDB7DEB7AB0150
:10161000BC0149835A836B837C830E94C70A49813A
:101620005A816B817C8188E090E00F900F900F9041
:101630000F90DF91CF910C94402FECE4F2E083E027
:10164000808310924D028FEF8283838314826081A6
:101650007181828193810C94010B80914C0280FFF7
:1016600003C086958F73089580E00895809150029D
:1016700090E001968430910514F083E090E080932F
:10168000500260914C0270914D0280914E029091F7
:101690004F020C94010B8091500290E0019797FF4C
:1016A00002C080E090E08430910514F083E090E087
:1016B0008093500260914C0270914D0280914E02D5
:1016C00090914F020C94010B8091710123E0829F55
:1016D000C00111248F5A9D4F6091020170E020914A
:1016E0004C0220FD0DC020E030E0F901EF5AFD4F23
:1016F0001182108212822D5F3F4F20333105A9F7EE
:101700000C94601190914C0290FF0FC020E030E0EB
:10171000F901EF5AFD4F8183608342832D5F3F4F74
:1017200020333105A9F70C94640B0895CF93DF9310
:1017300000D01F92CDB7DEB720914C0220FF0AC027
:101740009E012F5F3F4F0E94530A4B8169818A811E
:101750000E94820B0F900F900F90DF91CF91089510
:101760005F926F927F928F929F92AF92BF92CF9231
:10177000DF92EF92FF920F931F93CF93DF9300D0EE
:101780001F92CDB7DEB78C01E62EF42E522E80913B
:101790004C0280FF8BC0982F9E77923061F49E019F
:1017A0002F5F3F4FC8010E94530A4B8169818A8194
:1017B0000E94820B5BC0E82FE695EF739EE39E0FBD
:1017C0009F73943018F4F0904F0250C09AE39E0F2C
:1017D0009F73993068F4881F8827881F90914D0265
:1017E000292F220F022F082B97FB112710F93EC03B
:1017F00087E28E0F8F738A30C8F5F0E07997E0FDAD
:1018000002C021E001C02FEFEE7FEC59FC4F859123
:101810009491AC0184E0569547958A95E1F72403AD
:101820004001259F900C1124580188E9A81A8EEFD9
:10183000B80A91E5C92E92E0D92E28E6622E7724C7
:101840007394C501B3010E94A32E96014F2D6E2DF6
:101850000E94530AA80CB91C83E0C80ED11C81E871
:10186000C81682E0D80669F70E94640B80914C028A
:1018700000FB87F980934C02902F969580914D0242
:101880008078892B10FB87F980934D02E0924E02FD
:10189000F0924F02552051F060914C0270914D0230
:1018A00080914E0290914F020E94010B0F900F9079
:1018B0000F90DF91CF911F910F91FF90EF90DF90EC
:1018C000CF90BF90AF909F908F907F906F905F90E0
:1018D0000895282FECE4F2E09081991F9927991F31
:1018E00030914D02832F880F482F492B37FB552706
:1018F00050F9CA01089668E671E00E94B72E43814C
:1019000062810C94B00B81E00C94690C282F9091AB
:101910004C02991F9927991F30914D02832F880FF0
:10192000482F492B37FB552750F9CA01483051053C
:101930001CF4805A9E4F01C0089768E671E00E942F
:10194000B72E40914F0260914E020C94B00B81E093
:101950000C94860C60914E02262F30E0283F310512
:1019600014F4685F01C06FEF30914C02331F3327CE
:10197000331F90914D02592F550F97FB992790F9DE
:10198000282F40914F02852F832B0C94B00B81E0C0
:101990000C94AA0C60914E02262F30E028303105BD
:1019A00014F0685001C060E030914C02331F3327BF
:1019B000331F90914D02592F550F97FB992790F99E
:1019C000282F40914F02852F832B0C94B00B81E080
:1019D0000C94CA0C40914F02242F30E0283F31056F
:1019E00014F4485F01C04FEF30914C02331F33278E
:1019F000331F90914D02592F550F97FB992790F95E
:101A0000282F60914E02852F832B0C94B00B81E020
:101A10000C94EA0C40914F02242F30E0283031051D
:101A200014F0485001C040E030914C02331F33277E
:101A3000331F90914D02592F550F97FB992790F91D
:101A4000282F60914E02852F832B0C94B00B81E0E0
:101A50000C940A0D20E00C94B00BCF9390914C02A3
:101A600090FF40C09178811102C0926007C085321A
:101A700010F0986403C08F73880F982B90934C02DA
:101A8000662351F060914C0270914D0280914E029C
:101A900090914F020E94010BC0914C026C2F6695F1
:101AA0006F7370E04BE050E083E091E00E940D2FF7
:101AB000892B19F01092720103C081E080937201AA
:101AC000CC1FCC27CC1F90914D02892F880F97FBFC
:101AD000992790F940914F0260914E028C2BCF9143
:101AE0000C942A0DCF910895682F90914C029695F1
:101AF0009F7381E0890F853208F081E00C942D0DF1
:101B000081E00C94740D682F90914C0296959F7310
:101B10008FEF890F09F484E20C942D0D81E00C9471
:101B2000830D61E00C942D0DECE4F2E08081816086
:101B3000808386958F730C94910D60E00C942D0D2D
:101B400080917301811135C080911D028160809365
:101B50001D020E94AF1D811104C00E943C1E0E9404
:101B60001D0B0E94FD0A60934C0270934D028093FE
:101B70004E0290934F026E7761F40E941D0B0E94FB
:101B8000FD0A60934C0270934D0280934E02909335
:101B90004F020E94C70A81E08093720180914C023B
:101BA00080FF04C086958F730E949D0D81E0809315
:101BB00073010895ECE4F2E080818E7F8083608180
:101BC0007181828193810E94010B109272012FEF2B
:101BD00080E792E0215080409040E1F700C0000093
:101BE0000C94640B80914C0280FD0C94DA0D0C94E3
:101BF000940DCF93E82FF0E0E05AFC4FC491809110
:101C00006F01909170010E94631FEC2FF0E08E171E
:101C10009F0708F443C00E94571F90937001809360
:101C20006F0160916E0170E080E090E00E94942C62
:101C300020E030E04FE753E40E94B72B2BED3FE06C
:101C400049E450E40E94BD2D0E942A2E0E94312CAE
:101C50002BE43AE34EE25FE30E944A2B20EF3BEF96
:101C600048ED52E40E94BD2D0E94632C462F8091C6
:101C70004C02881F8827881F90914D02292F220F20
:101C800097FB992790F960914E02822B0E94960B48
:101C900080916E0190E0019680936E01CF9108953E
:101CA000CF93E82FF0E0E35AFC4FC49180916C0190
:101CB00090916D010E94631FEC2FF0E08E179F073B
:101CC000E8F00E94571F90936D0180936C01409142
:101CD0004F0260914E0280916A0190916B010E94C7
:101CE000960B80916A0190916B01019668E671E014
:101CF0000E94A32E90936B0180936A01CF91089567
:101D0000CF92DF92FF920F931F93CF93DF93F82E22
:101D1000E82FE695F0E0E65AFC4FC4918091680107
:101D2000909169010E94631FEC2FF0E08E179F07CE
:101D3000F0F10E94571F909369018093680101E5BB
:101D400012E0C0E0D0E088E6C82EDD24D394809174
:101D50006601909167018C0F9D1FB6010E94A32E12
:101D6000980140914F0260914E020E94530A66967C
:101D70000D5F1F4FC03681E0D80749F70E94640B02
:101D80002091660130916701F0FE0BC0C9010196F8
:101D900068E671E00E94A32E90936701809366012C
:101DA00006C0215031093093670120936601DF910D
:101DB000CF911F910F91FF90DF90CF900895AF9238
:101DC000BF92CF92DF92EF92FF920F931F93CF9328
:101DD000DF9380FF02C01FEF01C011E08695E82F5E
:101DE000F0E0E95AFC4FC491809164019091650143
:101DF0000E94631FEC2FF0E08E179F0708F465C068
:101E00000E94571F909365018093640121E5C22EC3
:101E100022E0D22E33E5E32E32E0F32EC0E0D0E014
:101E2000F70131971082F6011082F701108294E0D9
:101E3000A92EB12C00E080916301800F87FD805FA7
:101E4000082E000C990BC817D907E9F480914F02AE
:101E50008A9DA0018B9D500D112455954795559550
:101E6000479580914C02881F8827881F90914D02CA
:101E7000592F550F97FB992790F9960160914E02C3
:101E8000852B0E94530A010FF1E0AF1AB10899F6B1
:101E9000219683E0C80ED11CE3E0EE0EF11CC031A8
:101EA000D10509F0BDCF0E94640B80916301113010
:101EB00031F4811102C08FE006C0815004C090E06F
:101EC00001968F70992780936301DF91CF911F91C5
:101ED0000F91FF90EF90DF90CF90BF90AF9008955B
:101EE000EF92FF920F931F93CF93DF93E82FF0E0D1
:101EF000EC5AFC4FC49180916101909162010E9463
:101F0000631FEC2FF0E08E179F0708F464C00E9457
:101F1000571F909362018093610180E090E0FC0183
:101F2000EF5AFD4F11821082128203968033910581
:101F3000B1F781E5E82E82E0F82E03E512E0C0E07B
:101F4000D0E080916001082E000C990BC817D907CA
:101F5000ECF080910101082E000C990B8C179D0765
:101F6000ACF080914C02881F8827881F90914D0209
:101F7000592F550F97FB992790F9970140914F02E0
:101F800060914E02852B0E94530A07C0F8013197D9
:101F90001082F7011082F80110822196F3E0EF0E13
:101FA000F11C0D5F1F4FC031D10559F60E94640B23
:101FB0008091000190916001980F909360012091B1
:101FC0000101280F20930101121614F49F301CF018
:101FD000819580930001DF91CF911F910F91FF9028
:101FE000EF900895EF92FF920F931F93CF93DF939B
:101FF00080915E0190915F010E94631F883E934033
:10200000D0F10E94571F90935F0180935E01C091B1
:102010005C01D0915D012196C170DD27D0935D01F7
:10202000C0935C0181E5E82E82E0F82E10E008E71D
:10203000812F8695FE01E80FF11DCF018170992750
:10204000970140914F0260914E02FC010E9FC0012A
:102050000F9F900D11240E94530A1F5FF3E0EF0EB3
:10206000F11C103129F7DF91CF911F910F91FF9053
:10207000EF900C94640BDF91CF911F910F91FF9023
:10208000EF900895CF93DF9300D01F92CDB7DEB7C6
:1020900080915A0190915B010E94631FE2E5F3E099
:1020A0002591349182179307C0F1809159018111D4
:1020B0000CC09E012F5F3F4F4FEF6FEF80E090E02D
:1020C0000E94530A8A81809359010E94571F90935E
:1020D0005B0180935A0180915801813051F028F0C2
:1020E000823061F4409159010AC08091590140E069
:1020F00007C06091590140E080E003C040E080E00B
:1021000060E00E94820B8091580190E0019663E0AC
:1021100070E00E94B72E809358010F900F900F909F
:10212000DF91CF9108950F931F93CF93DF93809109
:102130005601909157010E94631F843F914008F41B
:1021400048C00E94571F9093570180935601C1E5E4
:10215000D2E000E010E020915401309155018091CF
:102160004C0290914D02083011051CF4232B79F09C
:1021700002C0232B61F4881F8827881F592F550F11
:1021800097FB992790F99E0140914F020AC0881F42
:102190008827881F592F550F97FB992790F99E0183
:1021A00040E060914E02852B0E94530A0F5F1F4F43
:1021B00023960031110579F60E94640B8091540139
:1021C00090915501019681709927909355018093C4
:1021D0005401DF91CF911F910F9108958091720169
:1021E0008823D9F190914C02892F86958F732EE325
:1021F000280F2F73243018F482500C94F90D2AE321
:10220000280F2F73233018F486500C94500E27E3B8
:10221000280F2F73263018F489500C94800E21E378
:10222000280F2F73263018F48F500C94DF0E2BE2FA
:10223000280F2F73233018F485510C94700F892FB9
:102240008E77803311F40C94F20F863411F40C94D1
:102250004210883411F40C94931008952EB1342F49
:10226000309523233EB1432B3FB7F894FC01680F10
:10227000791FE617F70789F0819198E04EB90000C1
:1022800000C087FF2EB9880F000000C000C000C04A
:102290002EB900C09A9591F7ECCF3FBF08952DB1AC
:1022A000242B2DB99B01220F331F620F731F0E9435
:1022B0002E1187EC90E00197F1F700C0000008951F
:1022C00044E00C944F119093790180937801089524
:1022D000E0917801F0917901309721F00190F0813F
:1022E000E02D099480E00895E0917801F091790162
:1022F000309799F020912001222359F020918702F4
:1023000027FF07C0DC012C9111962C93119725E033
:102310002C930280F381E02D09940895E0917801D7
:10232000F0917901309739F022E0DC012C930480A0
:10233000F581E02D0994089520917601309177017F
:102340008217930771F09093770180937601E09163
:102350007801F0917901309721F00680F781E02D26
:1023600009940895209174013091750182179307A3
:1023700071F09093750180937401E0917801F09170
:102380007901309721F00084F185E02D09940895BA
:1023900085B7806885BF85B7806885BF0895089533
:1023A00008950C94D01108950C94D3110E94C81173
:1023B0000E94CF110C94D11181E008950E944E1F0C
:1023C0000E9436090E9423200E9460230E94A00DD3
:1023D0000C94D4114F925F927F928F929F92AF9202
:1023E000BF92CF92DF92EF92FF920F931F93CF9302
:1023F000DF93CDB7DEB72A970FB6F894DEBF0FBED6
:10240000CDBF0E9480090E94DC11811111C08FEFA5
:1024100089838A831B820E94571F8160782F9D8346
:102420008C8349815A816B818D810E94A81257C08B
:102430009BE7C92E91E0D92E00E010E0AA24A394D6
:10244000B12C702E802F0E942C094C01F601419076
:1024500051906F01482659264114510431F40F5F01
:102460001F4F0530110569F7D2CF80911D0281FD04
:102470000E94350920E030E07501022E02C0EE0C0A
:10248000FF1C0A94E2F7C70184219521892B09F1E9
:102490002E837F828E209F2091E0892809F490E08E
:1024A00098870E94571F8160782F9A8789874E816D
:1024B0005F8168858A850E94A812000F111FF801AC
:1024C000E558FE4F80819181E826F926F182E0826D
:1024D00006C02F5F3F4F2F30310571F6C0CF0E94ED
:1024E000C62210917A010E9468111817D9F00E9433
:1024F000681180937A012A960FB6F894DEBF0FBE5A
:10250000CDBFDF91CF911F910F91FF90EF90DF90A2
:10251000CF90BF90AF909F908F907F905F904F90A3
:102520000C9402042A960FB6F894DEBF0FBECDBFFE
:10253000DF91CF911F910F91FF90EF90DF90CF909F
:10254000BF90AF909F908F907F905F904F90089535
:10255000CF93DF93CDB7DEB72B970FB6F894DEBFDE
:102560000FBECDBF4F83588769877A878B87DE017F
:10257000119686E0FD0111928A95E9F785E0FE014A
:10258000379601900D928A95E1F749815A816B81C6
:102590007C818D819E810E94F4192B960FB6F89450
:1025A000DEBF0FBECDBFDF91CF910895FC018081CA
:1025B00091810E94C01C0895882309F41AC18238B1
:1025C000C1F40E94681181FD14C169E380910E017C
:1025D00090910F010E94A31E0E944B1D2FEF81EED0
:1025E00094E0215080409040E1F700C0000069E392
:1025F00019C08338F9F40E94681180FDFAC063E5C0
:1026000080910E0190910F010E94A31E0E944B1D0C
:102610002FEF81EE94E0215080409040E1F700C020
:10262000000063E580910E0190910F010E94AE1EA3
:102630000C944B1D8438C1F40E94681182FDD9C0EE
:1026400067E480910E0190910F010E94A31E0E94E9
:102650004B1D2FEF81EE94E0215080409040E1F738
:1026600000C0000067E4DECF9CEF980F913A40F481
:10267000682F80910E0190910F010E94A31ED8CF68
:1026800090E2980F983050F4877091E001C0990F54
:102690008A95EAF7892F0E94021DCACF9BE5980F01
:1026A000933070F4853A29F0863A31F083E890E06F
:1026B00005C081E890E002C082E890E00C949C1193
:1026C00098E5980F973108F08EC0883A09F445C014
:1026D000893A09F445C08A3A09F445C08B3A09F4AD
:1026E00045C08C3A09F445C08B3B09F445C08C3B8E
:1026F00009F445C08D3A09F445C0803B09F445C052
:102700008E3A09F445C08F3A09F445C0813B09F47B
:1027100045C0823B09F445C0833B09F445C0843B76
:1027200009F445C0853B09F445C0863B09F445C022
:10273000873B09F445C0883B09F445C0893B09F44F
:1027400045C08D3B09F445C08E3B09F445C08A3B2A
:1027500009F445C080E090E044C082EE90E041C0C2
:1027600089EE90E03EC08AEE90E03BC085EB90E0C1
:1027700038C086EB90E035C083EB90E032C084EB4C
:1027800090E02FC087EB90E02CC08CEC90E029C04B
:102790008DEC90E026C083E891E023C08AE891E0C8
:1027A00020C082E991E01DC084E991E01AC081E275
:1027B00092E017C083E292E014C084E292E011C07C
:1027C00085E292E00EC086E292E00BC087E292E0E2
:1027D00008C08FE690E005C080E790E002C08AE282
:1027E00092E00C94B211803F20F00E94CE210C9414
:1027F000BB220895882309F464C0823879F40E94CA
:10280000681181FF5EC069E380910E0190910F0114
:102810000E94A31E0E944B1D69E310C08338B1F4CF
:102820000E94681180FF4DC063E580910E01909178
:102830000F010E94A31E0E944B1D63E580910E01B3
:1028400090910F010E94AE1E0C944B1D843879F4B8
:102850000E94681182FF35C067E480910E0190915B
:102860000F010E94A31E0E944B1D67E4E7CF9CEF5F
:10287000980F913A10F4682FE1CF90E2980F9830BA
:1028800050F4877091E001C0990F8A95EAF7892F7B
:102890000E94081DD9CF9BE5980F933020F480E06B
:1028A00090E00C949C1198E5980F973120F480E00B
:1028B00090E00C94B211803F20F00E9436220C94DC
:1028C000BB220895882321F00E94021D0C944B1D09
:1028D0000895882321F00E94081D0C944B1D089533
:1028E0004F925F926F927F92BF92CF92DF92EF9260
:1028F000FF920F931F93CF93DF937C01D62FC72FA7
:10290000FC01058102950F70128111110E941F1D9B
:102910000E94F81C882379F0112369F080E28D0F62
:10292000883048F082E00E94961D0E94F81C91E0D9
:10293000B82EB92601C0B12CCC2EC2948FE0C8228B
:10294000D12CF601E859FF4F0C94ED2E8C2F807F8F
:10295000CF70882311F0C295C07F112399F0CC234A
:1029600009F4D0C180E28D0F883010F0D11104C07D
:102970008C2F0E94021D03C08C2F0E94121D0E94EA
:102980004B1DC0C18D2F0E94FA13CC2309F403C242
:1029900080E28D0F883010F0D11104C08C2F0E947E
:1029A000081D03C08C2F0E94181D0E944B1DF3C1EF
:1029B0008C2F807FCF70803211F0C295C07FDD23D5
:1029C00019F0D130C9F022C0112371F0002341F079
:1029D000013031F40E94321D8C2B0E94381DDBC166
:1029E0000E94321D8C2B46C1002319F0013009F4DE
:1029F000D2C10E94411D18C0112321F0063008F0F9
:102A0000CAC10EC0053008F0C6C10EC0112351F076
:102A1000002331F0F701858180FF74C18F708583B9
:102A20008C2F28C101117FC18C2F2AC18C2F869534
:102A30008695837090E0009719F0019761F0ABC123
:102A4000112321F08D2F9C2F937002C080E090E025
:102A50000E949C11B0C1112321F08D2F9C2F9370E7
:102A600002C080E090E00E94B211A5C11123F9F0EC
:102A7000D53F51F0D63F71F0D43FA9F48091810247
:102A80009091820281600BC08091810290918202BC
:102A9000826005C08091810290918202846090934F
:102AA0008202809381028D2F0E94CE211EC0D53FCD
:102AB00051F0D63F71F0D43FA9F4809181029091FA
:102AC00082028E7F0BC080918102909182028D7F65
:102AD00005C080918102909182028B7F9093820247
:102AE000809381028D2F0E9436220E94BB2263C1F7
:102AF0008C2F837009F050C0111159C18D2F829510
:102B000086958770880F880F9D2F9F70492E512CB6
:102B1000612C712C082E04C0440C551C661C771CBB
:102B20000A94D2F7D4FF14C00FE010E020E030E0A8
:102B3000B901A80104C0440F551F661F771F8A956D
:102B4000D2F7CB01BA01609570958095909503C03E
:102B500060E070E0CB01C695C695C370D0E0C2308E
:102B6000D10561F0C330D10581F06429752986292A
:102B70009729219771F00E94391B19C16429752981
:102B8000862997290E944B1B12C10E94391BC30141
:102B9000B2010E94271B0BC1112319F08C2F8170E9
:102BA00001C08695882309F402C18D2F82958695F0
:102BB0008770880F880F9D2F9F70492E512C612C94
:102BC000712C082E04C0440C551C661C771C0A94FA
:102BD000D2F7D4FF14C00FE010E020E030E0B901DC
:102BE000A80104C0440F551F661F771F8A95D2F7AE
:102BF000CB01BA01609570958095909503C060E017
:102C000070E0CB01C695C695C3704C2F50E04230A2
:102C1000510569F04330510589F0642975298629E9
:102C200097294130510571F00E94FF1BC0C06429F3
:102C30007529862997290E94111CB9C00E94FF1B83
:102C4000C301B2010E94ED1BB2C08D2F90E0FC01C8
:102C5000E05EF109E531F10508F050C0E858FF4F9A
:102C60000C94ED2EDF708C2F8F71112331F00E94A8
:102C7000861B8D2F0E9462148EC00E94A71B8D2F71
:102C80000E94691488C0112341F0053008F083C008
:102C90008C2F8F710E94CC1B7EC0063008F07BC049
:102CA000F7CF112339F08C2F8F710E94861B73C0D0
:102CB0001123C9F38C2F8F710E94A71B6CC01123A5
:102CC00029F08C2F8F710E94711B65C00E946C1BB4
:102CD00062C0112349F0CF718C2F0E94861B63E0E4
:102CE0008C2F0E94811D57C081E00E94961D0230EA
:102CF00008F451C082E00E94961D4DC0112331F0AE
:102D0000002389F28D2F0E94DC1245C0002391F22E
:102D1000D93349F45FEF67EE73E051506040704083
:102D2000E1F700C000008D2F0E94FA1334C04C2F31
:102D30004F706D2FC7010E9479060E94981A3BC000
:102D4000111139C0CF70D0E0C230D10599F03CF4F8
:102D5000209769F02197F9F40E949A232CC0C4307F
:102D6000D10571F054F02597B1F480E00AC00E94BB
:102D70007D2321C00E94D9231EC00E94E0231BC0D6
:102D800085E00E94032417C04C2F4F706D2FC701A0
:102D90000E947C0610C088E0C816D10441F05CF0A7
:102DA000EAE0CE1AD108F2E0CF16D10420F40E9456
:102DB00068110E940204BB20F1F00E94F41C80FD07
:102DC0001AC0F70112820E94EE1C0E94861BC701E6
:102DD0000E9409170E94EE1CDF91CF911F910F9165
:102DE000FF90EF90DF90CF90BF907F906F905F90BB
:102DF0004F900C94A71BDF91CF911F910F91FF90E3
:102E0000EF90DF90CF90BF907F906F905F904F904A
:102E100008950F931F93CF93DF93EC0188819981DD
:102E20002B813C81232BB9F09F3F11F48F3F99F008
:102E3000CE010E941404882371F0688179818A810F
:102E40000E94CB1C8C010E94231C0E94241BB801F1
:102E5000CE010E947014DF91CF911F910F910895C0
:102E60000E941F1D0E942F1D0E944B1D0E94542373
:102E70000E94BB2280E090E00E949C1180E090E0E4
:102E80000C94B21180910E0190910F010E94B91E15
:102E90000C9430170E940F1D0C944217E92FE295F5
:102EA000EF70F0E03297EE30F105B0F4E357FF4FEA
:102EB0000C94ED2E803F91F018F4803E68F40EC023
:102EC000843F51F40BC0803E48F0813F29F406C096
:102ED00093FB882780F9089580E0089581E00895A4
:102EE0000E94C01C0E944E170895CF93DF9300D01C
:102EF00000D01F92CDB7DEB70F900F900F900F90BC
:102F00000F90DF91CF910895CF93DF9300D000D041
:102F100000D0CDB7DEB726960FB6F894DEBF0FBE51
:102F2000CDBFDF91CF9108951F93CF93DF93C091D1
:102F3000860116E080918701C81799F0D0E01C9FA8
:102F4000F0011D9FF00D1124E857FE4F4081518183
:102F500062817381848195810E9484172196C77054
:102F6000E9CFDF91CF911F9108954091B801509121
:102F7000B9016091BA017091BB018091BC0190913F
:102F8000BD010C9484178091BD0182958F7009F06A
:102F900054C08091BA01882309F44FC08091860102
:102FA000A09187016091B8017091B9014091BB0176
:102FB0005091BC01B6E08A1709F43FC090E041157A
:102FC0005105C1F17F3F11F46F3FA1F1B89FF001AE
:102FD000B99FF00D1124E857FE4F218172132AC0CA
:102FE0002081621327C02281211124C023813481D2
:102FF0002417350710F421503109241B350B283CC8
:103000003105C0F42091BD012F7020612093BD01D6
:1030100026E0289FF001299FF00D1124E357FE4F71
:1030200080818F708061808388EB91E00E94091716
:103030000C94941701968770BECF0895CF92DF92BB
:10304000EF92FF920F931F93CF93DF93CDB7DEB72D
:1030500062970FB6F894DEBF0FBECDBF8C0185E03E
:10306000F801DE011D9601900D928A95E1F7D801D5
:103070004C9111965C91119712966C911297139640
:10308000CD90DC9014973091B8017091B901809186
:10309000BB019091BC01009709F46BC17F3F19F40B
:1030A0003F3F09F466C1E090BA01EE2009F4C0C0C8
:1030B0002091BD01C816D90628F0F601E81BF90BCE
:1030C000CF0104C0809590958C0D9D1DFF24F39435
:1030D000883C910578F0F12C207F09F0C6C07C2D4A
:1030E000D98AC88A89890E94751788EB91E00E9465
:1030F0000917B1C0822F807F09F046C0751314C034
:10310000341312C0611110C02F7020612093BD01D3
:103110000E94B51788EB91E00E9409178091BD01CC
:10312000D80115968C932EC0CD2819F15F3F11F46C
:103130004F3FF9F0F62E61111CC08091860120915D
:10314000870136E0821709F45AC090E0389FF001F9
:10315000399FF00D1124E857FE4F7181571306C0B7
:103160007081471303C07281711103C0019687708B
:10317000E9CFF62E662309F427C18091BD01816055
:103180008093BD01F12C20C1751308C0341306C013
:10319000611104C08091BD01D801C3C04D875E8715
:1031A0008D859E856A8B0E9470176A898823E1F15C
:1031B0006623D1F12091BD01822F82958F7090E01E
:1031C000029774F08091B8019091B90198878F832C
:1031D0001986DB86CA862C87CE0107960E940917BE
:1031E00086E0F801A8EBB1E001900D928A95E1F735
:1031F0000E94C3170E94B517FF24F394E5C04D87C2
:103200005E878D859E850E94C01C292F22952F7078
:1032100030E0223031050CF0CBC09F7009F0C5C002
:10322000805E883008F4D0C0C8010E940917E4CF3E
:10323000C816D90608F453C0F601E81BF90BCF01F4
:10324000883C910508F450C0F12C7C2DD98AC88A9D
:1032500089890E947517E8EBF1E086E0DF011D9295
:103260008A95E9F70E94B517AFC0751314C03413DF
:1032700012C0611110C08091BD01F8018583C801A1
:103280000E94091786E0E8EBF1E0DF011D928A95C4
:10329000E9F7FE2C99C04D875E878D859E856A8BE8
:1032A0000E9470176A89882309F4BECF662309F447
:1032B000BBCF2091BD01822F82958F7090E0029745
:1032C0000CF48ECF8091B8019091B9019A838983D3
:1032D0001B82DD82CC822E83CE0101967FCF80952A
:1032E00090958C0D9D1DACCFF62E662309F49CCFD6
:1032F00075132EC034132CC02091BD0120FD1FC0BA
:10330000822F82958F70D9F0D80115962C9315973E
:103310008F3049F08F5F982F9295907F822F8F701A
:10332000892B15968C93C8010E94091786E0F80135
:10333000A8EBB1E001900D928A95E1F793CF86E07A
:10334000F801A8EBB1E001900D928A95E1F73CC03D
:103350004D875E878D859E850E947017811140CFB5
:103360008091BD0181608093BD01C8010E94091751
:103370002BC0662309F458CF4D875E878D859E85C7
:103380000E947017F82E882309F44ECF86E0F801CA
:10339000A8EBB1E001900D928A95E1F788EB91E0FE
:1033A0000E94D6120E94C3175DCF811139CF0CC085
:1033B000243031050CF038CF9F7009F431CFF8017B
:1033C0009581907F09F02CCF8F2D62960FB6F894DF
:1033D000DEBF0FBECDBFDF91CF911F910F91FF9048
:1033E000EF90DF90CF9008951F93CF93DF93CDB7E9
:1033F000DEB72C970FB6F894DEBF0FBECDBF4F835C
:10340000588769877A878B879C87CE0107960E94A9
:103410001E18882369F08F8198852A853B85232B88
:10342000F1F19F3F09F063C08F3F09F060C037C0E2
:1034300086E0FE013796DE01119601900D928A9585
:10344000E1F76F817885EA85FB85309741F17F3F11
:1034500011F46F3F21F12091870130E0C9010196FD
:10346000877099274091860150E08417950709F4E9
:1034700047C069837A83FD83EC8396E0929FD001F5
:10348000939FB00D1124A857BE4FFE0131960190B5
:103490000D929A95E1F7809387010E94941716E0A8
:1034A00080918601909187018917C1F1189FC00111
:1034B000112488579E4F0E941E18882379F1E091AD
:1034C00086011E9FF0011124E857FE4F4081518173
:1034D00062817381848195810E9484178091860125
:1034E00090E001968770992780938601D9CF4F810C
:1034F000588569857A858B859C850E948417CFCFF6
:103500000E944A171092870110928601E8EBF1E0C1
:1035100086E0DF011D928A95E9F7C1CF2C960FB6A0
:10352000F894DEBF0FBECDBFDF91CF911F910895FC
:10353000EF92FF920F931F93CF93DF938C01892B10
:1035400009F46CC0F12CEE24E394E8012196F80113
:103550008491843740F4843008F051C0813081F088
:10356000823019F15BC0853709F444C0A8F19CE7AB
:10357000980F903708F052C08F770E94FA1341C01D
:103580000E5F1F4FFE01C49180E28C0F883048F41B
:10359000C7708E2D01C0880FCA95EAF70E94221DC0
:1035A00014C08C2F0E94DC122DC00E5F1F4FFE0135
:1035B000C49180E28C0F883058F4C7708E2D01C002
:1035C000880FCA95EAF70E94281D0E944B1D1AC059
:1035D0008C2F0E94FA1316C00E5F1F4FFE01C4917C
:1035E000CC2381F08FE99FE00197F1F700C0000044
:1035F000C150F6CF0E5F1F4FFE01F49003C00E9432
:10360000DC128E018F2D882309F49FCFEFE9FFE0B4
:103610003197F1F700C000008150F5CFDF91CF91D5
:103620001F910F91FF90EF90089508950C94151B32
:103630000E94161B6093F4017093F5018093F601CC
:103640009093F7010C94301708950C94181B0F9366
:103650001F930091F4011091F5012091F601309132
:10366000F701602B712B822B932B1F910F910C94E0
:10367000181B0F931F930091F4011091F5012091F5
:10368000F6013091F70160237123822393231F9168
:103690000F910C94181B0F931F930091F40110913C
:1036A000F5012091F6013091F701602771278227FB
:1036B00093271F910F910C94181B08950C945D1B78
:1036C0000E945E1B6093F0017093F1018093F20100
:1036D0009093F3010C94301760E070E0CB010C94F0
:1036E000601B0F931F9341E050E060E070E08A019F
:1036F0009B0104C0000F111F221F331F8A95D2F7B0
:10370000C901B8011F910F910C94601B0F931F9377
:1037100041E050E060E070E004C0440F551F661FB8
:10372000771F8A95D2F78091F0019091F101A091D5
:10373000F201B091F3018A019B01082B192B2A2B6E
:103740003B2BC901B8011F910F910C94601B0F9383
:103750001F9341E050E060E070E004C0440F551F4B
:10376000661F771F8A95D2F74095509560957095A2
:103770008091F0019091F101A091F201B091F301DB
:103780008A019B01082319232A233B23C901B8017D
:103790001F910F910C94601B0F931F9341E050E019
:1037A00060E070E004C0440F551F661F771F8A95C4
:1037B000D2F78091F0019091F101A091F201B091C6
:1037C000F3018A019B01082719272A273B27C901F2
:1037D000B8011F910F910C94601B0F931F930091E0
:1037E000F0011091F1012091F2013091F301602B71
:1037F000712B822B932B1F910F910C94601B0F93B5
:103800001F930091F0011091F1012091F20130918C
:10381000F30160237123822393231F910F910C9452
:10382000601B0F931F930091F0011091F101209103
:10383000F2013091F30160277127822793271F91AE
:103840000F910C94601B08952FE0929F800D11241E
:10385000A82FA695A695A695877051E001C0550F93
:103860008A95EAF785E0A89FD001112420E030E096
:1038700070E0F901EA0FFB1FE254FE4F4081CB01DB
:10388000022E02C0969587950A94E2F781709927D7
:10389000819584278523842780832F5F3F4F2530A0
:1038A000310539F708952FE0929F800D1124682F7C
:1038B000669566956695982F977085E0689FB0012C
:1038C000112440E050E080E0FA01E60FF71FE254D7
:1038D000FE4F208130E0092E02C0369527950A94CC
:1038E000E2F721703327042E01C0220F0A94EAF771
:1038F000822B4F5F5F4F4530510531F70895BF92DE
:10390000CF92DF92EF92FF920F931F93CF93DF93AB
:103910008C01C090F401D090F501E090F601F09098
:10392000F7018091F0019091F101A091F201B09125
:10393000F301C82AD92AEA2AFB2ACFE1D0E0D7012D
:10394000C6010C2E04C0B695A795979587950A9445
:10395000D2F780FF07C0BC2EB8018C2F0E949706BB
:10396000019719F4219758F7B12C8B2DDF91CF9146
:103970001F910F91FF90EF90DF90CF90BF9008952F
:10398000CF93DF93EC010E947F1CBE010E9497063B
:10399000DF91CF9108951F93CF93DF93EB01909127
:1039A0008501992321F0CB010E94C01C13C08823FC
:1039B00049F0CB010E947F1C182F682FCE010E9476
:1039C000241C04C0CB010E94531C182FBE01812F60
:1039D0000E949706DF91CF911F9108958091F80181
:1039E00085958595859508958091F801877008954E
:1039F0009091F801977081E009F480E0089580913A
:103A00001C02089590911C02892B80931C0208953A
:103A1000809590911C02892380931C020895109236
:103A20001C02089590911B02892B80931B0208951C
:103A3000809590911B02892380931B020895109218
:103A40001B02089590911A02892B80931A020895FF
:103A5000809590911A02892380931A0208951092FA
:103A60001A0208958091F901089508950C94351D66
:103A70009091F901981721F08093F9010C94361D6B
:103A800008958091F901882329F01092F90180E0CE
:103A90000C94361D0895E0910E01F0910F01809174
:103AA0001C028083E0910E01F0910F0190818091C2
:103AB0001B02892B8083E0910E01F0910F01908110
:103AC00080911A02892B80838091F901882381F0EB
:103AD000E0910E01F0910F019081892B80838091FC
:103AE0000E0190910F010E943E1E81110E94411D06
:103AF00080910E0190910F010C94741108950C9413
:103B00007E1D98E0899F90011124262B2093F801B7
:103B10000E94861B8091F8018595859585950C946A
:103B20007F1D1092F80180E00C947F1D2091F80118
:103B3000809582238093F801982F977079F430E074
:103B4000482F082E000C550B2417350739F08595A2
:103B5000859585950E94A71B0C94911D089580E082
:103B600090E00E94282F21E08D3E9E4F09F020E03A
:103B7000822F089582E090E00C941A2F682F82E043
:103B800090E00C942E2F83E090E00C941A2F682F75
:103B900083E090E00C942E2F84E090E00C941A2F98
:103BA000682F84E090E00C942E2F86E090E00C9437
:103BB0001A2F682F86E090E00C942E2FAB01BC01E9
:103BC0008FE090E00C94402FAB01BC0183E190E0CA
:103BD0000C94402F60E070E0CB010C94E41D60E099
:103BE00070E0CB010E94DE1D0C94EA1D6DEE7EEFAD
:103BF00080E090E00E944C2F60E082E090E00E9424
:103C00002E2F60E083E090E00E942E2F1092F401AE
:103C10001092F5011092F6011092F70160E084E035
:103C200090E00E942E2F60E085E090E00E942E2F11
:103C300060E086E090E00E942E2F6FEF87E090E03A
:103C40000E942E2F40E050E0BA0188E090E00E94F0
:103C5000402F60E08DE090E00E942E2F40E050E089
:103C6000BA0188E190E00E94402F60E087E190E097
:103C70000E942E2F0C94EF1D0C94F61DFC01329621
:103C800080912001882331F08091870287FF02C054
:103C90009EE101C096E080E0915028F0219122231E
:103CA000D9F38F5FF9CF08959C01FC0132969FEF05
:103CB00080E04191461789F09F3F19F4411101C0FE
:103CC000982F8F5F8630A9F79F3F39F0F901E90FF0
:103CD000F11D97FDFA95628308950895FC013296CF
:103CE00008962081261301C010823196E817F90743
:103CF000C1F70895262F2695269526952E3168F42E
:103D0000FC01E20FF11D677021E030E001C0220FDD
:103D10006A95EAF78281282B22830895262F26951B
:103D2000269526952E3170F4FC01E20FF11D677087
:103D300021E030E001C0220F6A95EAF720958281E8
:103D400028232283089520912001222329F0209105
:103D5000870227FD0C947A1E0C94541E209120019A
:103D6000222329F02091870227FD0C948E1E0C94AB
:103D70006E1E20912001FC013296222331F08091A9
:103D8000870287FF02C08EE101C086E0DF011D923D
:103D90008A95E9F7089508950C94CB1E0E94CC1ED5
:103DA00080918E02843061F110921E0220E488E13D
:103DB00090E00FB6F894A895809360000FBE209312
:103DC000600080E00E948B0380E00E9402040E9459
:103DD000CC1E83B7817F846083BF83B7816083BF3C
:103DE0007894889583B78E7F83BF0FB6F894A89593
:103DF00080916000886180936000109260000FBE27
:103E0000089508950895CF930E94011F0E9480098C
:103E10000E94021FC0E08C2F0E942C09892B29F4DC
:103E2000CF5FC530C1F780E001C081E0CF91089538
:103E300008950C94181F0E944A170E9460230E9444
:103E400068110E9402040C94191F1F920F920FB662
:103E50000F9211248F939F93AF93BF9380911E0273
:103E6000811113C08091830290918402A0918502F8
:103E7000B09186024196A11DB11D8093830290935B
